:10000000000000308A006628A5002008840021092D
:10001000841780058413A50803192C28F030A70045
:1000200024088038A600F030A7030319A70003199D
:10003000A50303192C281C283020030128182108A7
:10004000A41F2108A40803190301A60F292880066C
:1000500010282A2800001328210884178004622809
:10006000290828040319A80A8030281AA906281983
:10007000A906A818A906290DA80DA90D2808622807
:10008000A501A400FF30A407031CA507031C6228D8
:100090000330A300DF304E204228A301E83EA20037
:1000A000A309FC30031C5728A20703185428A207F1
:1000B0000000A30F542822185D28A21C612800000C
:1000C000612808008313831203130800830145305D
:1000D000A8000330A900073083169F008501831212
:1000E0008501831686018312860183168701831298
:1000F00087010530A0001030A1003230A4003C3050
:100100008A0104204630A40014308A0104205530AE
:10011000A40078308A0104205330A40028308A01DA
:1001200004204630A40014308A0104203230A40098
:1001300014308A0104204630A40014308A010420BF
:100140005A30A40078308A0104205A30A4001430B8
:100150008A0104206230A400A0308A010420073004
:10016000A500D0308A0141208030AA000530A000CF
:100170001030A1002A08A40002308A0104200130B6
:10018000AA078A110A12031CB6280730A500D0302E
:100190008A0141200530A0001030A1002B30A400BE
:1001A00050308A0104203F30A40014308A0104201A
:1001B0004D30A40014308A0104204730A400503090
:1001C0008A0104203330A40014308A0104205A30FC
:1001D000A40014308A0104205530A4008C308A0118
:1001E00004204D30A40014308A0104205030A400B3
:1001F00014308A0104205530A40014308A010420F0
:100200005A30A40014308A0104205030A400143065
:100210008A0104205530A4003C308A0104205A3061
:10022000A4003C308A0104205C30A4003C308A01E8
:1002300004205730A4003C308A0104206030A40020
:1002400046308A010420A4010A308A01042060306B
:10025000A4000A308A010420A4010A308A01042083
:100260006030A4000A308A010420A4010A308A0107
:1002700004206030A4001E308A010420A4010A304A
:100280008A0104205C30A4001E308A010420A401ED
:100290000A308A0104205730A4001E308A0104204D
:1002A000A4010A308A0104206030A40028308A01A9
:1002B0000420A40114308A0104203F30A4000A3035
:1002C0008A010420A4010A308A0104203F30A400DE
:1002D0000A308A010420A4010A308A0104203F3038
:1002E000A4000A308A010420A4010A308A010420F3
:1002F0003F30A40014308A0104201730A50070306C
:100300008A0141208A0179288A0184298A01862963
:02400E00723FFF
:00000001FF
